:100000000C9462000C948A000C948A000C948A0070
:100010000C948A000C948A000C948A000C948A0038
:100020000C948A000C948A000C948A000C948A0028
:100030000C948A000C948A000C948A000C948A0018
:100040000C9496070C948A000C9464070C943E0759
:100050000C948A000C948A000C948A000C948A00F8
:100060000C94E0070C948A00000000002400270094
:100070002A000000000023002600290000000008DC
:10008000000201000003040700000000000000005F
:10009000040404040404040402020202020203032E
:1000A0000303030301020408102040800102040836
:1000B0001020010204081020000000002500280084
:1000C0002B00FF0811241FBECFEFD8E0DEBFCDBF4D
:1000D00012E0A0E0B1E0E2EDF2E202C005900D9284
:1000E000A035B107D9F723E0A0E5B2E001C01D9229
:1000F000A63FB207E1F710E0C2E6D0E004C02197C6
:10010000FE010E946111C136D107C9F70E9443095F
:100110000C9467110C9400002091420381E021327D
:1001200008F044C080911E038111FCCF80914103EF
:1001300092E090931E0391E090931D039FEF9093A4
:100140001C0310921B0320931A03A1E2B3E0EAEF11
:10015000F2E090E0291331C01092F9029091F90277
:10016000880F892B8093F9028091F802813049F53C
:100170001092F8028091F9028093BB008091BC003C
:1001800083FDF8CF85EC8093BC0080911E03823004
:10019000E1F380911C038F3FB1F080911C0380320A
:1001A000A1F080911C03803391F084E01092200331
:1001B0001092420310921F0308953D9131939F5F67
:1001C000C9CF85EEE0CF80E0F1CF82E0EFCF83E0D2
:1001D000EDCFCF93DF93AAEDB2E01196EC9111979A
:1001E000F0E0EE0FFF1FE854FF4FC591D4919FB789
:1001F000F8941092800088812C91822B88839FBF75
:1002000013961C921E921297DF91CF910895CF9270
:10021000DF92EF92FF92CF937C01BC01990F880B84
:10022000990B0E94F90F97012250310921333105B2
:1002300090F42AE939E949E15FE30E944F0F6B012D
:100240007C0120E030E0A9010E944A0F811120C00A
:1002500081E090E048C09701245331092C313105E9
:1002600068F420E030E040E250E40E944F0F20E0CC
:1002700030E040E852E40E94DE0EE1CF80E5E8166F
:10028000F10431F7C12CD12C80ECE82E82E4F82E59
:10029000CFB7F89483E6809380008BE18093810050
:1002A00089EF90E0909389008093880020E030E00F
:1002B00040E250E4C701B6010E94AE1020E030E0F9
:1002C00040E85FE30E94DD0E0E94C10F70938B0037
:1002D00060938A00CFBF81E090E09093DD0280932D
:1002E000DC0290E080E0CF91FF90EF90DF90CF9024
:1002F000089508950895AF92BF92CF92DF92EF9242
:10030000FF920F931F93CF93DF936C017B018B01BF
:10031000040F151FEB015E01AE18BF08C017D1070F
:1003200059F06991D601ED91FC910190F081E02D99
:10033000C6010995892B79F7C501DF91CF911F91EE
:100340000F91FF90EF90DF90CF90BF90AF90089506
:10035000FC01538D448D252F30E0842F90E0821BCB
:10036000930B541710F0CF96089501970895FC0150
:10037000918D828D981761F0A28DAE0FBF2FB11DA8
:100380005D968C91928D9F5F9F73928F90E0089500
:100390008FEF9FEF0895FC01918D828D981731F0BA
:1003A000828DE80FF11D858D90E008958FEF9FEF0E
:1003B0000895FC01918D228D892F90E0805C9F4FE4
:1003C000821B91098F739927089583E493E00E941B
:1003D000D90121E0892B09F420E0822F089580E0E3
:1003E00090E0892B29F00E94E50181110C94000016
:1003F0000895FC01A48DA80FB92FB11DA35ABF4FBA
:100400002C91848D90E001968F739927848FA68913
:10041000B7892C93A089B1898C91837080648C9367
:10042000938D848D981306C00288F389E02D808116
:100430008F7D80830895EF92FF920F931F93CF9348
:10044000DF93EC0181E0888F9B8D8C8D98131AC00F
:10045000E889F989808185FF15C09FB7F894EE89F6
:10046000FF896083E889F989808183708064808353
:100470009FBF81E090E0DF91CF911F910F91FF909E
:10048000EF900895F62E0B8D10E00F5F1F4F0F7346
:100490001127E02E8C8D8E110CC00FB607FCFACF01
:1004A000E889F989808185FFF5CFCE010E94F901A5
:1004B000F1CFEB8DEC0FFD2FF11DE35AFF4FF082D2
:1004C0009FB7F8940B8FEA89FB8980818062CFCF38
:1004D000CF93DF93EC01888D8823B9F0AA89BB897B
:1004E000E889F9898C9185FD03C0808186FD0DC066
:1004F0000FB607FCF7CF8C9185FFF2CF808185FF87
:10050000EDCFCE010E94F901E9CFDF91CF9108959F
:10051000833081F028F4813099F08230A9F0089579
:100520008730A9F08830C9F08430B1F48091800020
:100530008F7D03C0809180008F7780938000089525
:1005400084B58F7784BD089584B58F7DFBCF80916E
:10055000B0008F778093B00008958091B0008F7DB8
:10056000F9CFCF93DF93EEE7F0E08491E6EAF0E095
:10057000D491E2E9F0E0C491CC23A1F081110E9472
:100580008802EC2FF0E0EE0FFF1FEE58FF4FA59111
:10059000B491EC91ED2381E090E009F480E0DF91EB
:1005A000CF91089580E090E0FACF1F93CF93DF932F
:1005B000282F30E0F901E458FF4F8491F901EC5500
:1005C000FF4FD491F901E057FF4FC491CC23A9F01C
:1005D000162F81110E948802EC2FF0E0EE0FFF1F12
:1005E000E854FF4FA591B4918FB7F894EC91111195
:1005F00008C0D095DE23DC938FBFDF91CF911F9190
:100600000895DE2BF8CF1092D9021092D8021092E2
:1006100020031092420310921E0381E080931D0379
:100620001092F80261E082E10E94D50261E083E16C
:100630000E94D502E9EBF0E080818E7F808380818B
:100640008D7F808388E48093B80085E48093BC002C
:1006500089E791E09093D7028093D6028AE791E0F0
:100660009093D5028093D4020895CF93DF9390E0C6
:10067000FC01EC55FF4F249180579F4FFC01849162
:100680008823D1F090E0880F991FFC01E859FF4FB3
:10069000A591B491FC01E854FF4FC591D49162300B
:1006A00071F49FB7F8943C91822F809583238C93AB
:1006B000E8812E2B28839FBFDF91CF9108958FB7BC
:1006C000F894EC912E2B2C938FBFF6CF3FB7F89474
:1006D0008091BC029091BD02A091BE02B091BF0278
:1006E00026B5A89B05C02F3F19F00196A11DB11D8D
:1006F0003FBFBA2FA92F982F8827BC01CD01620FC9
:10070000711D811D911D42E0660F771F881F991F83
:100710004A95D1F708958F929F92AF92BF92CF9250
:10072000DF92EF92FF924B015C010E9466036B0126
:100730007C010E9466036C197D098E099F09683E41
:10074000734081059105A8F321E0821A9108A10860
:10075000B10888EEC80E83E0D81EE11CF11C81149C
:100760009104A104B10429F7FF90EF90DF90CF909E
:10077000BF90AF909F908F9008950895CF92DF9291
:10078000EF92FF920F931F938FB7F894C090C0021F
:10079000D090C102E090C202F090C3028FBF0091DE
:1007A000B3021091B4022091B5023091B602C01A82
:1007B000D10AE20AF30A6091B7027091B8028091FF
:1007C000B9029091BA0248EEC41643E0D406E1049F
:1007D000F10438F41F910F91FF90EF90DF90CF90CC
:1007E00008956F5F7F4F8F4F9F4F6093B702709355
:1007F000B8028093B9029093BA0208511C4F2F4F50
:100800003F4F0093B3021093B4022093B50230938C
:10081000B602BACF85ED8093BC008091BC0084FD08
:10082000FCCF10921E03089520919002260F3327CB
:10083000331F21323105ECF420911E03FC0190E0BE
:1008400080E0243069F082E00895A0919002219127
:10085000AC0140595D4FA40FB52FB11D2C930196EB
:10086000861798F380919002680F6093900280E061
:10087000089581E008950895E091D9028091D80209
:10088000E81730F4F0E0E05BFD4F808190E00895E0
:100890008FEF9FEF08959091D9028091D8022FEFAA
:1008A0003FEF981748F4E92FF0E0E05BFD4F20811F
:1008B00030E09F5F9093D902C90108958091D802DA
:1008C0009091D902891B990B0895CF92DF92EF92F4
:1008D000FF920F931F93CF93DF937C01CB018A018B
:1008E00020911F03222389F0EB016B01C40ED51E5A
:1008F000CC15DD0569F06991D701ED91FC9101906E
:10090000F081E02DC7010995F3CF642F0E941404F4
:10091000C801DF91CF911F910F91FF90EF90DF9071
:10092000CF900895CF93DF931F92CDB7DEB7698341
:1009300020911F032223F9F020914203203258F026
:1009400021E030E0FC013383228390E080E00F90CF
:10095000DF91CF91089580912003E82FF0E0EF5DC3
:10096000FC4F998190838F5F809320038093420393
:1009700081E090E0ECCF61E0CE0101960E9414048A
:10098000F7CF6295607F4111616021116460FC01C5
:10099000258121116860FC01848191E090931F03FF
:1009A00080934103109220031092420380EE93E063
:1009B0000E9492040C948C0090E080E0089560E026
:1009C00088E00C94D50290E080E00C94C70E61E0C2
:1009D00088E00E9435030E94DF041092E802109222
:1009E000E9020E94E304813208F080E29AE0E8E440
:1009F000F1E0AEEDB2E001900D929A95E1F786300C
:100A000008F486E08093EF0261E08AE00E943503FB
:100A1000EEEAF0E0E491E093DA02EAE9F0E0E49152
:100A2000E093DB020C94E9000F931F93CF93DF93C5
:100A3000EC01162F042F21E00E94C10420E0402F7A
:100A4000612FCE010E94C1048FE890E00197F1F779
:100A5000DF91CF911F910F9108950F931F93CF9323
:100A6000DF938C01C62FD42F62956F700E941405FE
:100A70006C2F6F704D2FC801DF91CF911F910F9197
:100A80000C94140541E00E942D0581E090E008954A
:100A9000CF93DF93CDB7DEB728970FB6F894DEBFBC
:100AA0000FBECDBF98E0E0E4F1E0DE0111960190C9
:100AB0000D929A95E1F79091F503691710F06FEF99
:100AC000690F262F30E0220F331F41E050E04C0F1A
:100AD0005D1F240F351FF9016081680F606840E0D9
:100AE0008CEE93E028960FB6F894DEBF0FBECDBF14
:100AF000DF91CF910C942D0540E061E08CEE93E006
:100B00000E942D058BE39FE10197F1F708950F9364
:100B10001F93CF93DF938B01877098E0899FB0017B
:100B20001124606440E08CEE93E00E942D05E80102
:100B3000085F1F4F69918CEE93E00E944205C01739
:100B4000D107C1F7DF91CF911F910F910895FB015C
:100B500001900020E9F73197AF01461B570BDC01EC
:100B6000ED91FC910280F381E02D09948F929F9288
:100B7000AF92BF92EF92FF920F931F93CF93DF93A9
:100B8000CDB7DEB7A1970FB6F894DEBF0FBECDBFCD
:100B90007C01FA01CB0119A2223008F42AE08E016F
:100BA0000F5D1F4F822E912CB12CA12CBF01A501EE
:100BB00094010E942011F901CA016A300CF5605DB0
:100BC000D8016E938D01232B242B252B79F790E0F0
:100BD00080E0109721F0BD01C7010E94A705A196F2
:100BE0000FB6F894DEBF0FBECDBFDF91CF911F913E
:100BF0000F91FF90EF90BF90AF909F908F900895CE
:100C0000695CDECF482F50E070E060E02AE08CEEB7
:100C100093E00C94B605CF92DF92EF92FF920F9380
:100C20001F93CF93DF936B01770FEE08FF08F7FE5A
:100C30001FC0EC01E881F9810190F081E02D6DE2A7
:100C400009958C0144275527BA014C195D096E0995
:100C50007F092AE0CE010E94B605800F911FDF9127
:100C6000CF911F910F91FF90EF90DF90CF9008955B
:100C70002AE0B701A601DF91CF911F910F91FF905C
:100C8000EF90DF90CF900C94B6054F925F926F92E9
:100C90007F928F929F92AF92BF92CF92DF92EF920C
:100CA000FF920F931F93CF936B017C01742EAC01C5
:100CB0009B010E941B1162E871E0811126C0460170
:100CC0005701E894B7F82FEF3FEF4FE75FE7C50113
:100CD000B4010E941B1181110CC02FEF3FEF4FE7B1
:100CE0005FE7C501B4010E944A0F66E871E018167B
:100CF00064F02FEF3FEF4FE75FE4C701B6010E94BA
:100D0000A9101816ACF46AE871E08CEE93E0CF916C
:100D10001F910F91FF90EF90DF90CF90BF90AF9019
:100D20009F908F907F906F905F904F900C94A7054D
:100D30002FEF3FEF4FE75FECC701B6010E944A0F6C
:100D400087FDE1CF20E030E0A901C701B6010E9494
:100D50004A0F10E000E087FF0CC041E06DE28CEE2E
:100D600093E00E942D05F7FAF094F7F8F09401E073
:100D700010E0C0E060E070E080E09FE37C1641F0AE
:100D800020E030E040E251E40E944F0FCF5FF6CF09
:100D9000A70196010E94DE0E4B015C010E94C80F64
:100DA0002B013C012AE0BC01A2018CEE93E00E94E1
:100DB000B605080F191FCC23D9F1C301B2010E9457
:100DC000F70F9B01AC01C501B4010E94DD0E4B0180
:100DD0005C0141E06EE28CEE93E00E942D050F5F16
:100DE0001F4FC15028F120E030E040E251E4C5013E
:100DF000B4010E94AE102B013C010E94C80F4B01B0
:100E0000B12CA12C2AE0B501A4018CEE93E00E9444
:100E1000B605080F191FC501B4010E94F70F9B0109
:100E2000AC01C301B2010E94DD0E4B015C01D9CFC0
:100E3000C801CF911F910F91FF90EF90DF90CF905D
:100E4000BF90AF909F908F907F906F905F904F90EA
:100E50000895CF93DF93BC0183E493E00E94A7053C
:100E6000EC016EE871E083E493E00E94A7058C0F2B
:100E70009D1FDF91CF9108950C94A7051F920F92AB
:100E80000FB60F9211242F933F934F935F936F935D
:100E90007F938F939F93AF93BF93EF93FF9383E4DD
:100EA00093E00E94F901FF91EF91BF91AF919F9163
:100EB0008F917F916F915F914F913F912F910F9003
:100EC0000FBE0F901F9018951F920F920FB60F92A2
:100ED00011242F938F939F93EF93FF93E0915303EC
:100EE000F09154038081E0915903F0915A0382FDFF
:100EF0001BC0908180915C038F5F8F7320915D0395
:100F0000821741F0E0915C03F0E0ED5BFC4F958FC0
:100F100080935C03FF91EF919F918F912F910F90A0
:100F20000FBE0F901F9018958081F4CF1F920F92E3
:100F30000FB60F9211242F933F938F939F93AF93EC
:100F4000BF938091C0029091C102A091C202B09162
:100F5000C3023091BB0223E0230F2D3758F50196D1
:100F6000A11DB11D2093BB028093C0029093C102CA
:100F7000A093C202B093C3028091BC029091BD02C3
:100F8000A091BE02B091BF020196A11DB11D809338
:100F9000BC029093BD02A093BE02B093BF02BF916A
:100FA000AF919F918F913F912F910F900FBE0F9016
:100FB0001F90189526E8230F0296A11DB11DD2CFD0
:100FC0001F920F920FB60F9211242F933F934F93BE
:100FD0005F936F937F938F939F93AF93BF93EF93A1
:100FE000FF938091B900887F803609F44AC0F0F5FC
:100FF000883209F4A7C018F5803109F49BC0B8F411
:10100000882309F4F9C0883009F494C0FF91EF9166
:10101000BF91AF919F918F917F916F915F914F9110
:101020003F912F910F900FBE0F901F901895883110
:1010300009F488C0803251F780931C0314C08034B7
:1010400009F49DC040F48033B9F38833F9F68093F6
:101050001C0385ECB0C0803509F485C0883509F4DF
:1010600096C0883499F60E940A04D0CF883909F4D2
:101070008CC038F5883729F050F4883611F0803765
:1010800029F683E080931E031092B20257C088387D
:1010900009F47BC0803919F0803809F0B7CF80910E
:1010A000B202803208F071C0E091B20281E08E0F8E
:1010B0008093B2028091BB00F0E0EE56FD4F80833A
:1010C0003DC0803B39F0E0F4803A09F479C0883AB9
:1010D00009F09CCF84E080931E031092910210923D
:1010E0009002E091D602F091D7020995809190028A
:1010F00081110FC081E0809390021092700209C0AC
:10110000803C09F4A6CF883C09F4A3CF883B09F0C2
:101110007DCFE091910281E08E0F80939102F0E00B
:10112000E059FD4F80818093BB00909191028091A6
:10113000900229C08091F9028093BB0085EC8093D6
:10114000BC0064CF90911B0380911A03981758F547
:10115000E0911B0381E08E0F80931B03F0E0E650CB
:10116000FD4F8081E9CFE0911B0381E08E0F8093DA
:101170001B038091BB00F0E0E650FD4F808390910F
:101180001B0380911A039817C8F285E8D8CFE09125
:101190001B0381E08E0F80931B038091BB00F0E066
:1011A000E650FD4F808380911D0381115CCF81E06B
:1011B0008093F80284EA8093BC0010921E0326CF2D
:1011C00085EC8093BC0010921E038091B2028032A5
:1011D00030F4E091B202F0E0EE56FD4F10826091E3
:1011E000B20270E0E091D402F091D50282E992E07F
:1011F00009951092B2020ACF10921C0334CFE3E497
:10120000F3E01382128288EE93E0A0E0B0E08483E2
:101210009583A683B78326E531E03183208325ECCF
:1012200030E03587248724EC30E03787268720ECB0
:1012300030E0318B208B21EC30E0338B228B22ECA1
:1012400030E0358B248B26EC30E0378B268B118EEB
:10125000128E138E148EE0EEF3E0138212828483DA
:101260009583A683B78388E691E091838083ECEE33
:10127000F3E0138212828AE791E09183808387E210
:10128000848315820895789484B5826084BD84B582
:10129000816084BD85B5826085BD85B5816085BD71
:1012A00080916E00816080936E0010928100809129
:1012B00081008260809381008091810081608093B1
:1012C0008100809180008160809380008091B100D6
:1012D00084608093B1008091B00081608093B00001
:1012E00080917A00846080937A0080917A00826095
:1012F00080937A0080917A00816080937A00809157
:101300007A00806880937A001092C100E0915303C4
:10131000F091540382E08083E0915303F0915403F1
:101320001082E0914F03F09150031082E09151033D
:10133000F091520380E1808310925B03E0915703A8
:10134000F091580386E08083E0915503F0915603B5
:10135000808180618083E0915503F0915603808104
:1013600088608083E0915503F09156038081806806
:101370008083E0915503F091560380818F7D8083B7
:1013800081E991E00E94290788E991E00E942907FC
:101390000E94030381E080931F0387E2809341034F
:1013A00010922003109242030E948C00C82FD0E0BC
:1013B0006CEA71E083E493E00E943C07BE0183E4A1
:1013C00093E00E940B0684EB91E0CD2B11F081ECB1
:1013D00091E00E94290782ED91E00E94290712E026
:1013E0001093F50388E08093F2030E94030320E04A
:1013F00040E060E08CEE93E00E94C1048BE39DE04E
:101400000197F1F740E063E08CEE93E00E94140551
:10141000CBE4D6E4CE010197F1F740E063E08CEE37
:1014200093E00E9414052197F1F740E063E08CEE11
:1014300093E00E94140583E592E00197F1F740E004
:1014400062E08CEE93E00E9414056091F20360620A
:1014500040E08CEE93E00E942D0584E08093F3033E
:1014600040E06CE08CEE93E00E942D050E947C052C
:101470001093F40340E066E08CEE93E00E942D05AB
:101480008FEF8093F10320E041E060E08CEE93E089
:101490000E94C1040E94E704C091E80262E082E079
:1014A0000E9435030E94E304D82F0E94B102892BC9
:1014B00009F069C08091DC029091DD02019709F486
:1014C00062C08091E8028D7F843009F45CC00E9484
:1014D000B102892B09F050C0D03238F5DF5F0E948D
:1014E0007C0561EE71E08CEE93E00E943C0761E0C8
:1014F00080E00E94480561EF71E08CEE93E00E946D
:101500003C0761E08DE00E9448058D2F0E94020695
:101510006FEF71E08CEE93E00E943C0768E572E0AB
:1015200080E090E00E948B03D2CF0E947C0561EEA8
:1015300071E08CEE93E00E943C0761E080E00E9445
:10154000480561EF71E08CEE93E00E943C0761E09A
:101550008DE00E94480586E00E9402066FEF71E070
:101560008CEE93E00E943C0768E572E080E090E03A
:101570000E948B03D6E0ABCF6D2F90E080E00E94FD
:10158000CF0E0E94E7040E94B102892B09F06FC0C0
:101590008091E802833009F06AC00E94E9006CE2A1
:1015A00071E080E090E00E948B030E947C0561E086
:1015B00072E08CEE93E00E943C070E94E3040E94DC
:1015C00002066FEF71E08CEE93E00E943C0761E051
:1015D00080E00E9448056CE072E08CEE93E00E948F
:1015E0003C0770E060E08CEE93E00E940B066EE03A
:1015F00072E08CEE93E00E943C076CE072E08CEEAF
:1016000093E00E943C0770E060E08CEE93E00E9463
:101610000B066EE072E08CEE93E00E943C076CE0FB
:1016200072E08CEE93E00E943C0770E060E08CEE8C
:1016300093E00E940B066DEF71E08CEE93E00E9448
:101640003C076091CC027091CD028091CE029091C6
:10165000CF0241E00E94450660E172E08CEE93E02B
:101660000E943C070E94DF0486E08093E80264E663
:1016700070E04FEF53E090E080E021E420937C00A5
:1016800020917A00206420937A0020917A0026FD30
:10169000FCCF2091780030917900821793070CF4E9
:1016A00047C1241735070CF4A9016150710929F7C6
:1016B0002091DC023091DD022130310541F420918E
:1016C000E6023091E7024217530708F04FC120911C
:1016D000DE023091DF028217930708F049C12091A2
:1016E000E0023091E1028217930708F423C1809150
:1016F000E802863009F082E0C817C1F09091EA0252
:10170000891709F439C19FB7F8944091C0025091EC
:10171000C1026091C2027091C3029FBF4093EB026D
:101720005093EC026093ED027093EE028093EA0214
:101730008091E802C81739F0813009F047C10E9452
:10174000DF040E94E900C093E9028091E80283303F
:1017500009F0D0C08091F0029091F102A091F202C4
:10176000B091F3028093F4029093F502A093F602F5
:10177000B093F7020E94BE030091C4021091C5020B
:101780002091C6023091C702601B710B820B930B34
:101790006093F0027093F1028093F2029093F3024F
:1017A0000E94BE030091C4021091C5022091C6029E
:1017B0003091C702601B710B820B930B6093D002B8
:1017C0007093D1028093D2029093D30220E831E546
:1017D00041E050E00E94421120E13EE040E050E054
:1017E0000E94421149012CE330E040E050E00E94A9
:1017F000421129016B018901EB0161E080E00E9447
:1018000048058AE08816910434F46CE072E08CEEAE
:1018100093E00E943C07B4018CEE93E00E940B061B
:101820006EE072E08CEE93E00E943C070A301105F6
:1018300034F46CE072E08CEE93E00E943C07B2015D
:101840008CEE93E00E940B066EE072E08CEE93E06B
:101850000E943C072A9734F46CE072E08CEE93E02F
:101860000E943C07B6018CEE93E00E940B066DEFE0
:1018700071E08CEE93E00E943C076091D002709181
:10188000D1028091D2029091D3020E94F70F6B0196
:101890007C0120E030E046E653E46091C80270919C
:1018A000C9028091CA029091CB020E94AE109B01A6
:1018B000AC01C701B6010E94AE1020E030E041E665
:1018C00055E40E944F0F20E030E04AE754E40E94C4
:1018D0004F0F6093CC027093CD028093CE02909311
:1018E000CF0241E00E94450660E172E08CEE93E099
:1018F0000E943C078091E8029091E902891759F013
:10190000833009F416C208F08EC0813009F496C005
:10191000823009F466C180E090E0892B09F4BCCDE7
:101920000E94E501882309F4B7CD0E940000B4CDE0
:10193000C901BBCE2091E2023091E30282179307E6
:1019400038F08091E802863009F4D6CE83E0D4CE18
:101950002091E4023091E5022817390758F480916C
:10196000E802863009F4C8CE84E0C6CE85E0C4CE55
:1019700081E0C2CE80E0C0CE9FB7F8944091C00213
:101980005091C1026091C2027091C3029FBF009149
:10199000EB021091EC022091ED023091EE02401B1F
:1019A000510B620B730B0AEF10E020E030E0813046
:1019B00021F409E110E020E030E040175107620710
:1019C000730708F4B3CE8093E802B0CE863009F4F2
:1019D000B6CE823041F40E94DF048091EF0290E0A5
:1019E0000E940701B0CE8330A1F48091EF0290E015
:1019F0000E94070161E088E00E94D5020E94BE03B8
:101A00006093C4027093C5028093C6029093C7028C
:101A10009ACE843009F493CE8530E9F20E94E90031
:101A20000E94DF0490CE843009F4ACC1853009F007
:101A300072CF0E947C056FE372E0CEC01092D0029C
:101A40001092D1021092D2021092D3021092CC02C4
:101A50001092CD021092CE021092CF020E947C050D
:101A600068E371E081E00E94870560E080E00E9409
:101A7000480561E08CEE93E00E94420560E371E06E
:101A800082E00E94870560E081E00E94480562E0F4
:101A90008CEE93E00E94420560E082E00E944805DF
:101AA00064E172E08CEE93E00E943C0768E271E032
:101AB00083E00E94870560E083E00E94480563E0C0
:101AC0008CEE93E00E94420560E271E084E00E94A7
:101AD000870560E084E00E94480564E08CEE93E0B6
:101AE0000E94420568E171E085E00E94870560E0A0
:101AF00085E00E94480565E08CEE93E00E94420577
:101B000060E171E086E00E94870560E086E00E9467
:101B1000480566E08CEE93E00E94420568E071E0C3
:101B200087E00E94870560E087E00E94480567E043
:101B30008CEE93E00E94420560E088E00E94480538
:101B400063E08CEE93E00E94420560E071E088E083
:101B50000E94870560E089E00E94480568E08CEEFD
:101B600093E00E94420560E08AE00E94480566E931
:101B700071E08CEE93E00E943C0760E08BE00E94F5
:101B8000480568E08CEE93E00E94420560E08CE03E
:101B90000E94480561E08CEE93E00E94420560E0FF
:101BA0008DE00E94480566E08CEE93E00E944205BD
:101BB00061E080E00E94480561EF71E08CEE93E007
:101BC0000E943C0761E08DE00E9448050E94E3040A
:101BD0000E9402066FEF71E08CEE93E00E943C07DA
:101BE0009ACE0E947C058091D0029091D102A09162
:101BF000D202B091D302892B8A2B8B2B31F466E170
:101C000072E08CEE93E00E943C078091D0029091AC
:101C1000D102A091D202B091D302892B8A2B8B2BB7
:101C200009F479CE60E272E08CEE93E00E943C070A
:101C300068E072E08CEE93E00E943C070E94E304AF
:101C40000E9402066FEF71E08CEE93E00E943C0769
:101C500061E080E00E9448056091D0027091D1025D
:101C60008091D2029091D30220E831E541E050E02A
:101C70000E94421120E13EE040E050E00E9442110B
:101C800049012CE330E040E050E00E94421129017C
:101C90006B018901EB0161E080E00E9448059AE058
:101CA0008916910434F46CE072E08CEE93E00E94AB
:101CB0003C07B4018CEE93E00E940B066EE072E0EC
:101CC0008CEE93E00E943C070A30110534F46CE07E
:101CD00072E08CEE93E00E943C07B2018CEE93E040
:101CE0000E940B066EE072E08CEE93E00E943C07CF
:101CF0002A9734F46CE072E08CEE93E00E943C078B
:101D0000B6018CEE93E00E940B066DEF71E08CEE55
:101D100093E00E943C076091CC027091CD028091CB
:101D2000CE029091CF0241E00E94450660E172E050
:101D300053CF0E947C0568E272E08CEE93E00E9433
:101D40003C0768E072E08CEE93E00E943C070E9442
:101D5000E3040E9402066FEF71E08CEE93E00E94B4
:101D60003C070E94E304682F70E090E080E00E944E
:101D7000F70F6093C8027093C9028093CA029093D0
:101D8000CB02C9CD0E947C0561E372E025CFF999B1
:101D9000FECF92BD81BDF89A992780B50895262F70
:101DA000F999FECF1FBA92BD81BD20BD0FB6F89440
:101DB000FA9AF99A0FBE019608955058BB27AA27A0
:101DC0000E94F50E0C946F100E94611038F00E9472
:101DD000681020F039F49F3F19F426F40C945E103B
:101DE0000EF4E095E7FB0C945810E92F0E94801048
:101DF00058F3BA17620773078407950720F079F440
:101E0000A6F50C94A2100EF4E0950B2EBA2FA02D7F
:101E10000B01B90190010C01CA01A0011124FF2797
:101E2000591B99F0593F50F4503E68F11A16F04092
:101E3000A22F232F342F4427585FF3CF4695379591
:101E40002795A795F0405395C9F77EF41F16BA0B56
:101E5000620B730B840BBAF09150A1F0FF0FBB1F04
:101E6000661F771F881FC2F70EC0BA0F621F731F4D
:101E7000841F48F4879577956795B795F7959E3FAA
:101E800008F0B0CF9395880F08F09927EE0F97953B
:101E9000879508950E94341008F481E008950E9407
:101EA000630F0C946F100E94681058F00E9461102C
:101EB00040F029F45F3F29F00C94581051110C9414
:101EC000A3100C945E100E94801068F39923B1F364
:101ED000552391F3951B550BBB27AA276217730750
:101EE000840738F09F5F5F4F220F331F441FAA1FE4
:101EF000A9F335D00E2E3AF0E0E832D091505040A0
:101F0000E695001CCAF72BD0FE2F29D0660F771F4D
:101F1000881FBB1F261737074807AB07B0E809F033
:101F2000BB0B802DBF01FF2793585F4F3AF09E3FB8
:101F3000510578F00C9458100C94A3105F3FE4F313
:101F4000983ED4F3869577956795B795F7959F5FFB
:101F5000C9F7880F911D9695879597F90895E1E047
:101F6000660F771F881FBB1F621773078407BA07A6
:101F700020F0621B730B840BBA0BEE1F88F7E09501
:101F800008950E94C80F6894B1110C94A31008958D
:101F90000E94881088F09F5798F0B92F9927B75161
:101FA000B0F0E1F0660F771F881F991F1AF0BA95FD
:101FB000C9F714C0B13091F00E94A210B1E00895A9
:101FC0000C94A210672F782F8827B85F39F0B93F9B
:101FD000CCF3869577956795B395D9F73EF49095B0
:101FE0008095709561957F4F8F4F9F4F0895E8942E
:101FF00009C097FB3EF490958095709561957F4F51
:102000008F4F9F4F9923A9F0F92F96E9BB279395FE
:10201000F695879577956795B795F111F8CFFAF40E
:10202000BB0F11F460FF1BC06F5F7F4F8F4F9F4F3F
:1020300016C0882311F096E911C0772321F09EE89D
:10204000872F762F05C0662371F096E8862F70E003
:1020500060E02AF09A95660F771F881FDAF7880FDD
:102060009695879597F90895990F0008550FAA0B33
:10207000E0E8FEEF16161706E807F907C0F012169B
:102080001306E407F50798F0621B730B840B950B9E
:1020900039F40A2661F0232B242B252B21F40895F3
:1020A0000A2609F4A140A6958FEF811D811D089590
:1020B00097F99F6780E870E060E008959FEF80ECFB
:1020C000089500240A94161617061806090608959E
:1020D00000240A9412161306140605060895092E04
:1020E0000394000C11F4882352F0BB0F40F4BF2B73
:1020F00011F460FF04C06F5F7F4F8F4F9F4F0895B3
:1021000057FD9058440F551F59F05F3F71F04795A8
:10211000880F97FB991F61F09F3F79F0879508958D
:10212000121613061406551FF2CF4695F1DF08C0AC
:10213000161617061806991FF1CF869571056105C9
:1021400008940895E894BB2766277727CB0197F971
:1021500008950E94341008F48FEF08950E94C11072
:102160000C946F100E94611038F00E94681020F0EB
:10217000952311F00C9458100C945E1011240C94BB
:10218000A3100E94801070F3959FC1F3950F50E04B
:10219000551F629FF001729FBB27F00DB11D639F19
:1021A000AA27F00DB11DAA1F649F6627B00DA11DBF
:1021B000661F829F2227B00DA11D621F739FB00D65
:1021C000A11D621F839FA00D611D221F749F3327D5
:1021D000A00D611D231F849F600D211D822F762F6E
:1021E0006A2F11249F5750409AF0F1F088234AF04B
:1021F000EE0FFF1FBB1F661F771F881F91505040B7
:10220000A9F79E3F510580F00C9458100C94A31030
:102210005F3FE4F3983ED4F3869577956795B7953D
:10222000F795E7959F5FC1F7FE2B880F911D969557
:10223000879597F908950E943410880B990B08959B
:10224000A1E21A2EAA1BBB1BFD010DC0AA1FBB1FBA
:10225000EE1FFF1FA217B307E407F50720F0A21B2C
:10226000B30BE40BF50B661F771F881F991F1A9499
:1022700069F760957095809590959B01AC01BD01C3
:10228000CF010895052E97FB1EF400940E9459116A
:1022900057FD07D00E94201107FC03D04EF40C9488
:1022A000591150954095309521953F4F4F4F5F4FB5
:1022B000089590958095709561957F4F8F4F9F4FB2
:1022C0000895EE0FFF1F0590F491E02D0994F89406
:0222D000FFCF3E
:1022D20011111915131111000E04040404040E0047
:1022E2001F040404040404001111111111110E0041
:1022F2001010101010101F000E11111111110E00EC
:1023020011111111110A04001F10101E10101F00CC
:1023120000004000140054006C030D03B2020000E0
:102322000401000000001B027B01A8016802D90120
:10233200B701CB010000000092046504DC043B04F9
:102342005E044B043C040000000042057B01DC04F7
:10235200BD036E616E00696E66006F7666000D0ADF
:10236200004C43442E2E2E00446F73653A2063685E
:1023720065636B20666F72204C4344004572726F36
:10238200723A20003A204C434420666F756E642EE8
:10239200003A204C4344206E6F7420666F756E6461
:1023A2002E0045562D4F4C5554494F4E2E4E4554F6
:1023B20000534554204D41582043555252454E54E6
:1023C200004D41582043555252454E543A20004147
:1023D2000053544F505045442040200030003A00F2
:1023E2006B5768002D00434F4E4E45435445440001
:1023F20043484152474544004348415247494E47AA
:102402000056454E542052455155495245440044C8
:10241200494F44452043484B204641494C454400DE
:00000001FF
